:03000000022EB518
:0C2EB50078FFE4F6D8FD75816E022EFC5B
:100EC30020000A3C2E2E2E3E004950436F6E6E6565
:100ED30063745245510A004950436F6E6E656374E3
:100EE300000A49504E6F41434B210A003E432C56A2
:100EF3002C43432CC0E4E0EFF2E5F020D1E8EDEA27
:100F0300EEEC49500A003E432C4D41432C25303230
:100F130062583A25303262583A25303262583A25BF
:100F2300303262583A25303262583A2530326258AC
:100F33002C4D414320E0E4F0E5F10A003E432C56FA
:100F430045522C20332E3220EEF2202573202573B8
:100F53002CC2E5F0F1E8FF20495020ECEEE4F3EB7E
:100F6300FF0A004E6F7620313920323031300031A4
:100F7300363A34393A3333003E432C4C442C5052E6
:100F83004F473A20202020202020202020202020EE
:100F9300202020202020202020202020202020204E
:100FA300202020202020202020202020202020203E
:100FB300202020202020202020202020202020202E
:100FC30020202020202020202CC4E0F2E020EFF07D
:100FD300EEF8E8E2EAE828F4E0E9EB290A003E2A21
:100FE3002C312CCEF1EDEEE2EDFBE520EFE0F0E06D
:100FF300ECE5F2F0FB20F1E5F2E5E2EEE3EE20E8CA
:10100300EDF2E5F0F4E5E9F1E00A003E412C413070
:10101300312C2562752E2562752E2562752E25626B
:10102300752C495020E0E4F0E5F120E0E4E0EFF234
:10103300E5F0E00A003E412C4130322C2562752E4A
:101043002562752E2562752E2562752C495020E088
:10105300E4F0E5F120EEF1ED2E20F1E5F0E2E5F02C
:10106300E00A003E412C4130332C2562752E256267
:10107300752E2562752E2562752C495020E0E4F00B
:10108300E5F120F0E5E72E20F1E5F0E2E5F0E00AF6
:10109300003E412C4130342C2562752E2562752E7D
:1010A3002562752E2562752CCCE0F1EAE020F1E58E
:1010B300F2E80A003E412C4130352C2562752E257D
:1010C30062752E2562752E2562752CD8EBFEE70A14
:1010D300003E2A2C312CC4EEEF2E20EFE0F0E0ECA2
:1010E300E5F2F0FB20F1E5F2E5E2EEE3EE20E8EDD8
:1010F300F2E5F0F4E5E9F1E00A003E422C53303129
:101103002C2562752CC6E4E0F2FC20E7E0EFF0EE5C
:10111300F1E020F1EEE5E4E8EDE5EDE8FF20EEF2A5
:1011230020F1E5F0E2E5F0E00A003E422C533032D4
:101133002C2562752CCEE1ECE5ED20F120F1E5F0F4
:10114300E2E5F0EEEC20E1E5E720EAE2E8F2E0EDAB
:10115300F6E8E90A003E422C5330332C2562752C05
:10116300CFE5F0E5E7E0EFF3F1EA20EFF0E820EF79
:10117300EEF2E5F0E520F1E2FFE7E820F120F1E50A
:10118300F0E2E5F0EEEC0A003E454E440A000A4464
:10119300756D7058202020202030302030312030D1
:1011A3003220303320303420303520303620303771
:1011B3002030382030392030412030422030432045
:1011C3003044203045203046000A3A003A20000AD5
:1011D300000A44756D7044202020202030302030D8
:1011E3003120303220303320303420303520303637
:1011F3002030372030382030392030412030422011
:101203003043203044203045203046004572722060
:101213006B657900526420656570726F6D0A0052C8
:1012230064204D454D0A00526420436F64650A00F3
:10123300577269746520436F64650A00446562757B
:10124300674950204F4E0A00446562756749502034
:101253004F46460A00446562756755736572204FB1
:101263006E0A00446562756755736572204F464682
:101273000A0044656275674D7367204F6E0A004428
:10128300656275674D7367204F46460A00436F6E6C
:10129300666967206C6F636B210A0057722065656E
:1012A30070726F6D0A0020536176652065657072F8
:1012B3006F6D210A00457272204D414321004C6F2E
:1012C30061643E3E002A003C4130313D003C4130E8
:1012D300323D003C4130333D003C4130343D003C25
:1012E3004130353D003C21003C5330313D003C53FF
:1012F30030323D003C5330333D003C5330353D00EC
:061303003C5330363D00B2
:0638AA00016B0001690042
:10390C00C28E438910E4F58B758DB8D2ABD28E2262
:03001B00022E258D
:102E2500C0E0C083C082C0D0C28E758B00758DB8DE
:102E3500201D0675A61E75A6E10569D219E56B600C
:102E450002056BE56AD394014002156A056EE56ECD
:102E5500540F7048D225E56E543F7012D217906614
:102E65008BE0600A04F0E0D394B44002D21D906672
:102E750086E0600204F0906104E0600214F0906660
:102E85008CE0D394014003E014F0301C02056CE59E
:102E95006DD394644004D21D8002056DE568D3941A
:102EA5000140021568D28ED0D0D082D083D0E032D6
:10086900C291C290D2B5C2227D027C007F071238A4
:100879008D8F49E549646060097D017F601237E821
:10088900D222E4FDFC7F0B12388D8F49E54930E611
:10089900097D04E4FF12380CD2227D017C007F0718
:1008A90012388D8F49E5497008FD7FFF1237E8D26C
:1008B90022302203126000C288C2A8C2AA75890028
:1008C90012334F90633EE0B4FA06A3E064CE607B36
:1008D900E4F54974362549F582E43463F583E4F097
:1008E9000549E549B443EC90633E74FAF0A374CE2C
:1008F900F0A374CCF0906344740AF0E4A3F0A30469
:10090900F0A3F090633A74FFF0A3F0A3F0E4A3F02E
:10091900906355740AF0E4F549E5492401FFE4338D
:10092900FE74362549F582E43463F583E0FD123718
:10093900C40549E549C3944340DFE4F5A775A61EFC
:1009490075A6E1907FF0F0A3F080FE9063497403EF
:10095900F0A374CCF0E4906348F0122B36C2B512C0
:10096900304DC21D1235DCD222C224C223906576D5
:100979007408F09062B47424F0E4A3F090633EE04C
:100989009062B6F090633FE09062B7F0906340E008
:100999009062B8F0906341E09062B9F0906342E0F0
:1009A9009062BAF0906343E09062BBF0756A01E42B
:1009B900906577F0C21EC21FC220C221202218AF43
:1009C90049FE7D031228B6E4FF122D7C7E0E7FC3FB
:1009D900E4FBFDFC1227B690668BE060037401F01E
:1009E900E4906104F0F56C906575F0F56D12390CC1
:1009F90075A70775A61E75A6E1D2AFE4F56D9061DE
:100A090004E070031225AA90668CE06401701D90C1
:100A190080007410F09080A874FFF0A3F0A3F0A3F5
:100A2900F0E490668CF0D222C223C224908008E0C0
:100A3900F54930E405D21E7410F0E54930E508D2D5
:100A4900209080087420F0E54930E608D21F908094
:100A5900087440F0E56CC394034019908002E4F0F7
:100A6900908001F0908000F0E56C94064006E4F572
:100A79006C1235DC9080A0E070031234479080B886
:100A8900E070031233CD9080D0E07003123580906E
:100A99008000E07013301E101226B2906331EFF01F
:100AA900D394004003120026908002E070069080E3
:100AB90000E06005D21C020A04C21CE4F56C9061D6
:100AC90004E06003020A04202212906578E0600CB9
:100AD9007E0E7FC5122A64E4906578F030201212E8
:100AE90021FC906331EFF0D394004005E0FF120040
:100AF90021201F03020C7A121EFF906331EFF07060
:100B090003020A04906375E054BF247F7003020B4B
:100B1900E3147003020BBB24026003020C1C2022A5
:100B2900077E0E7FCC122A64202603020C7A90637A
:100B39004DE07006906351E06067906682E0FF9037
:100B4900634DE0B50724906683E0FE90634EE0B5FF
:100B59000618906684E0FE90634FE0B5060C906637
:100B690085E0FE906350E06E6037906351E06F60FE
:100B790003020C7A906683E0FF906352E06F600392
:100B8900020C7A906684E0FF906353E06F60030281
:100B99000C7A906685E0FF906354E06F6003020C65
:100BA9007AC21A9065777401F012001E756A010203
:100BB9000C7A90668BE060037401F090667AE0FF2E
:100BC900906377E06F6003020C7A90667AE004F034
:100BD900E4F56A906575F0020C7A301A03020C7A12
:100BE900906344E07003020A04906355740AF0129A
:100BF9003830D21AE4F56A906575F090668604F08B
:100C0900E4906679F0A3F02022677E0E7FDA122A3B
:100C190064805E90668BE060037401F0301A529034
:100C29006375E020E74B906377E0FF906679E0FE1B
:100C39006F600D906681E07007EE146F703380135A
:100C4900906679E004F0906331E0FFD394044003A7
:100C59001236369060007482F0A37401F0906377C5
:100C6900E0906002F07E607F007D03123251020A3B
:100C790004201A03020D92E56A7068123792EF6038
:100C8900237E647F75906476E02404FD12325190CE
:100C99006681E07009906355E0F56A020A04E4F59B
:100CA9006A020A04906686E0D3943C4036906681D5
:100CB900E0703090668604F0122CC7E4906475F0F9
:100CC900A37412F090667AE0906477F0A374FDF053
:100CD90090610563A20190647963A2017F12121CDD
:100CE9004D809E1239278F49E549B401159060005E
:100CF9007483F0E4A3F07E607F007D02123251021A
:100D09000A04E549D39401401C9060007483F0A360
:100D19007401F0E54924FEA3F07E607F007D031293
:100D29003251020A04E56A64016003020A0490650B
:100D390075E004F02022077E0E7FE4122A64906396
:100D490055E0C394C85004E02432F0906575E0C3BF
:100D59009405400DC21AE4906577F012001E020A4C
:100D6900047C667D82906349E0FAA3E0FB7F02126E
:100D79002FC97E647F75906476E02404FD12325198
:100D8900906355E0F56A020A04E56A6401600302AA
:100D99000A04906577E014604624FE6042147003EB
:100DA900020E8524046003020A04E4F56C2026136C
:100DB9009065777404F0906575E05401F0756A01E7
:100DC900020A049080027410F0E4906577F090654F
:100DD9007504F0756AFA90668274FFF0020A04904D
:100DE9006682E07003020E6F9064757480F09064FF
:100DF900777401F0E4A3F0A304F0A37430F0A374B2
:100E09007BF0E4F549747C2549F582E43464F58383
:100E1900747DF0747D2549F582E43464F583E4F04A
:100E2900E5492407906476F07C667D82906349E009
:100E3900FAA3E0FB7F02122FC97E647F75E549247E
:100E490009FD123251906681E0601B123830D21AC6
:100E5900E4F56A906575F090668604F0E490667929
:100E6900F0A3F0020A04302607E4906577F08006C3
:100E79009065777404F0756AFA020A049080027426
:100E890010F0756A05906575E06401FFF09065776B
:100E99007401F0EF7012906351E0600C12177590B5
:100EA900668212178D020A0490634D1217759066B7
:090EB9008212178D020A0480FE6A
:010EC200220D
:10002600906376E0B444047F0180027F009063759C
:10003600E0B447047E0180027E00EE5F604A906372
:100046003EE0906377F090633FE0906378F09063D2
:1000560040E0906379F0906341E090637AF09063BA
:1000660042E090637BF0906343E090637CF09063A2
:10007600767452F09062AE63A2019080A863A201EA
:100086007F06121C4D02085F906331E0C39408504E
:100096000302086890633EE0FF906377E06F6003B9
:1000A60002086890633FE0FF906378E06F600302A8
:1000B6000868906340E0FF906379E06F6003020890
:1000C60068906341E0FF90637AE06F60030208681E
:1000D600906342E0FF90637BE06F600302086890E4
:1000E6006343E0FF90637CE06F60030208689063FF
:1000F60076E06444701A9080A8E0B4FF139062AE74
:1001060063A2019080A863A2017F06121C4D801095
:100116009062B2E09080ACF09062B3E09080ADF077
:1001260090668BE060037401F090668C7464F090C6
:1001360063767452F0906375E0646D600302026941
:100146007BFF7A0E79EF12136B7BFF7A0F7909909A
:10015600633EE0F552A3E0F553A3E0F554A3E0F5C2
:1001660055A3E0F556A3E0F55712136B7552FF75CC
:10017600530F7554667555FF75560F7557727BFF8D
:100186007A0F793F12136B7BFF7A0F797B12136B11
:100196007BFF7A0F79E112136B7BFF7A10790E9051
:1001A6006344E0F552A3E0F553A3E0F554A3E0F56C
:1001B6005512136B7BFF7A10793890634DE0F55238
:1001C600A3E0F553A3E0F554A3E0F55512136B7BBA
:1001D600FF7A107966906351E0F552A3E0F553A3D8
:1001E600E0F554A3E0F55512136B7BFF7A10799472
:1001F60090633AE0F552A3E0F553A3E0F554A3E08B
:10020600F55512136B7BFF7A1079B7906336E0F5DC
:1002160052A3E0F553A3E0F554A3E0F55512136B92
:100226007BFF7A1079D412136B7BFF7A1079FDA2CB
:1002360026E433F55212136B7BFF7A11792D906603
:1002460081E0F55212136B7BFF7A11795890668B19
:10025600E0F55212136B122F417BFF7A11798B1244
:10026600136B22906375E0644C70737E117F91FB73
:10027600FDFC1227B690637DE0F54AA3E0F54BE45A
:10028600F54DE54A90637FF0A3E54BF07E117FCCF8
:100296007C637D7F7B021227B6E4F54C854B828515
:1002A6004A83E0FF747F254CF582E43463F583EFDF
:1002B600F0054BE54B7002054A054CE54CB410DCE5
:1002C6007E117FCF7C637D7F7B101227B6054DE5BF
:1002D6004DC3941040AC7E117FD2122A64229063E3
:1002E60075E0646C7060F54E7E117FD4FBFDFC12E8
:1002F60027B6E4F54DE490637FF0A3E54EF07E115A
:100306007FCC7C637D7F7B021227B6E4F54CA84E3A
:10031600E6FF747F254CF582E43463F583EFF00540
:100326004E054CE54CB410E67E117FCF7C637D7F95
:100336007B101227B6054DE54DC3940840B77E11D4
:100346007FD2122A6422906375E0644B7061F54C8B
:100356007467254CF582E43463F583E06032746794
:10036600254CF582E43463F583E0F4602374672555
:100376004CF582E43463F583E0FF747D254CF58209
:10038600E43463F583E0B50710054CE54CB408C0CA
:100396009061047432F002085F9063757421F03046
:1003A600220302085F7E127F0F122A6402085F9002
:1003B6006375E0B4521A2022077E127F17122A6450
:1003C6009063757472F07E637F757D081231D12259
:1003D600906375E0644970452022077E127F2212E1
:1003E6002A6490637DE0F54AA3E0F54BE4F54C857D
:1003F6004B82854A83E0FF747F254CF582E43463A3
:10040600F583EFF0054BE54B7002054A054CE54CCC
:10041600B480DC7E637F757D8A1231D1229063754C
:10042600E0644370462022077E127F2A122A6490D7
:10043600637DE0F54AA3E0F54BE4F54C854B8285F8
:100446004A83E493FF747F254CF582E43463F58395
:10045600EFF0054BE54B7002054A054CE54CB480C0
:10046600DB7E637F757D8A1231D122906375E064ED
:100476005A70532022077E127F33122A6490637DBE
:10048600E0F54AA3E0F54B7C637D7F7B80AF4BAE06
:100496004A12375EE4F54C854B82854A83E493FF26
:1004A600747F254CF582E43463F583EFF0054BE564
:1004B6004B7002054A054CE54CB480DB7E637F75C4
:1004C6007D8A1231D122906375E06444600302058F
:1004D6005D90637DE0FF6444700302085FEFB43112
:1004E6000CC2227E127F3F122A6402085F90637D4F
:1004F600E0B4300CD2227E127F4B122A6402085FCF
:1005060090637DE0B4320CD2237E127F58122A64A7
:1005160002085F90637DE0B4330CC2237E127F66CF
:10052600122A6402085F90637DE0B4340CD2247E04
:10053600127F75122A6402085F90637DE0B4350C61
:10054600C2247E127F82122A6402085F90637DE0D5
:10055600FF12002202085F906104E0701320220758
:100566007E127F90122A649063757421F002085FF0
:100576009061047432F0906375E0FFB45104C2AF29
:1005860080FEEF645770452022077E127F9E122A56
:100596006490637EE0906331F0E4F54C906331E063
:1005A600FFE54CC39F400302085F747F254CF5822C
:1005B600E43463F583E0FF90637DE0254C24ADF5DC
:1005C60082E43461F583EFF0054C80D0906375E0EA
:1005D600645360030206802022077E127FA9122A36
:1005E6006490633EE0FF9061B6E06F703C90633FBD
:1005F600E0FF9061B7E06F7030906340E0FF90617C
:10060600B8E0B50724906341E0FF9061B9E0B50713
:1006160018906342E0FF9061BAE0B5070C9063431F
:10062600E0FF9061BBE06F60169063757421F03057
:10063600220302085F7E127FB8122A6402085FE472
:10064600F54CE4F56DAF4CFE74AD254CF582E43403
:1006560061F583E0FD1237C4054CE54CC394FE40BA
:10066600E1C2AFE4907FF0F0A3F0907FFD74AAF0B2
:10067600A374FFF0A37455F080FE906375E0644F99
:10068600704C90637DE0F54AA3E0F54BE54B454A97
:10069600700A2022077E127FC1122A642022077E5A
:1006A600127FC8122A64E4F54C747F254CF582E467
:1006B6003463F583E0854B82854A83F0054BE54B31
:1006C6007002054A054CE54CB480DE02085F906373
:1006D60075E0FFB4452190637DE0FDA3E0907FF0D7
:1006E600CDF0A3EDF0C2AF907FFD74AAF0A374FF26
:1006F600F0A37455F080FEEF64656003020868900D
:10070600637DE0FFA3E0907FF0CFF0A3EFF0E4F588
:100716004AF54BD3907FF1E0954B907FF0E0954AF8
:100726004020E4F56D254BFFE54A3401FE854B82FA
:10073600854A83E0FD1237C4054BE54B7002054A36
:1007460080D17E127FCA123151EF4E602012000313
:10075600906344EFF0120003906345EFF01200033C
:10076600906346EFF0120003906347EFF07E127F2E
:10077600D0123151EF4E602012000390634DEFF01E
:1007860012000390634EEFF012000390634FEFF0F8
:10079600120003906350EFF07E127FD6123151EFB4
:1007A6004E6020120003906351EFF0120003906335
:1007B60052EFF0120003906353EFF01200039063C0
:1007C60054EFF07E127FDC123151EF4E60201200A2
:1007D6000390633AEFF012000390633BEFF01200D0
:1007E6000390633CEFF012000390633DEFF07E123E
:1007F6007FE2123151EF4E6020120003906336EF14
:10080600F0120003906337EFF0120003906338EFA5
:10081600F0120003906339EFF0E4F54CE4F56DE572
:100826004C2401FFE433FE7436254CF582E4346330
:10083600F583E0FD1237C4054CE54CC3944340DC18
:10084600C2AFE4907FF0F0A3F0907FFD74AAF0A30E
:1008560074FFF0A37455F080FE7E637F757D0812E9
:0208660031D18E
:01086800226D
:10372600AE07EEC39430400BEED394395005EE2429
:10373600D0FF22EEC39461400BEED394665005EEA3
:1037460024A9FF22EEC39441400BEED394465005C4
:08375600EE24C9FF22AF062298
:1038E2009062ACE475F0011216659062ACE0FEA342
:0638F200E0FF1238702215
:100003001238E2123726EFC454F0FEC0061238E26B
:08001300123726D0E02FFF2276
:10352300E4906C8CF01238E2906C8DEFF0C3943021
:103533004018E0FFD394395011906C8CE02405F5CA
:1035430082E43461F583EFF08011906C8CE0240504
:10355300F582E43461F583E4F0800C906C8CE00434
:10356300F0E0D3940840BE754D00754E00754F00D2
:0C357300E4F5507B017A617905121D5BC4
:01357F002229
:043151008E4F8F50BE
:103155009062ACE4F0A374FFF01238E2EF6069F41A
:103165006066855082854F83E493B507EC75510100
:10317500E5502551F582E4354FF583E493602590BC
:1031850062ADE02551FF9062ACE03400FE1238706C
:10319500E5502551F582E4354FF583E493B50704F1
:1031A500055180CCE5502551F582E4354FF583E492
:1031B5009370A6E55124FFFFE434FF9062AC8FF0D5
:0B31C5001216657E007F0122E4FEFF71
:0131D00022DC
:102B36007E127FE8123151EF4E70037F01227E1222
:102B46007FEB123151EF4E600C1238E2EF24D024A5
:102B5600FF92268002D2267E127FF1123151EF4E6D
:102B6600600C1238E2EF24D0906681F08005E49084
:102B76006681F07E127FF7123151EF4E600C1238EB
:102B8600E2EF24D090668BF08005E490668BF07EB1
:102B9600127FFD123151EF4E600C1238E2EF24D055
:102BA60024FF92188002C21890633E63A2019066C9
:102BB6007B63A2017F06121C4D30183B7E137F03F8
:102BC600123151EF4E603012000390667BEFF01227
:102BD600000390667CEFF012000390667DEFF01222
:102BE600000390667EEFF012000390667FEFF0120E
:0A2BF6000003906680EFF07F0022DC
:1036DD00906576E0C3947C40027F0A906576E0FEAB
:1036ED0004F074B42EF582E43462F583EFF0BF0A72
:1036FD0027906576E0FF04F074B42FF582E4346210
:10370D00F583E4F0906576E0FF1232D19065767422
:09371D0008F09062B5E004F0220E
:1035DC009080007480F090633663A201F583F582CD
:1035EC0063A2017F08121C4D90633E63A201908080
:1035FC008863A2017F0A121C4D9080927407F0A37D
:10360C0074D0F0A37406F0906348E0FF9080B1F0A2
:10361C009080E1EFF09080957455F0A3F0908000CD
:0A362C007401F090800974F0F022A0
:10344700908009E04410F09080A0E070609080A127
:103457007482F09080A874FFF0A3F0A3F0A3F07F2C
:10346700039080AEEFF0A374CBF09080007402F06D
:10347700906C8012179900000000906C80E090809B
:1034870040F0906C81E0908041F0906C82E09080F9
:1034970042F0906C83E0908043F0A3E4F0A3F0A3A4
:0D34A700F0A3F0908018F0A3F0A3F0A3F0C4
:0134B40022F5
:10358000908009E04440F09080D17482F07F0390F5
:1035900080DEEFF0A374CCF09080027402F0906CA7
:1035A0008412179900000000906C84E0908058F01D
:1035B000906C85E0908059F0906C86E090805AF095
:1035C000906C87E090805BF0A3E4F0A3F0A3F0A3FD
:0B35D000F0908030F0A3F0A3F0A3F017
:0135DB0022CD
:1033CD00908009E04420F09080B8E0706C9080B956
:1033DD007482F07F039080C6EFF07FCDA3EFF07F76
:1033ED00039080C4EFF0A374CDF09080C074FFF013
:1033FD00A3F0A3F0A3F09080017402F0906C8812FA
:10340D00179900000000906C88E090804CF0906C53
:10341D0089E090804DF0906C8AE090804EF0906C39
:10342D008BE090804FF0A3E4F0A3F0A3F0A3F09015
:09343D008024F0A3F0A3F0A3F039
:013446002263
:102FC9008C4A8D4BA907EAFDE975F018A424ACFFDA
:102FD900E5F034808F82F583EDF0EBFDE975F018AB
:102FE900A4FFAEF024ACFBEE34808B82F583A3ED15
:102FF900F0854B828C83E0FDEF24A8FFEE3480FE40
:103009008F82F583EDF0854B828C83A3E08F828ECE
:1030190083A3F0854B82854A83A3A3E0FDE975F07C
:1030290018A424A8FFE5F03480FE8F82F583A3A3BA
:10303900EDF0854B828C83A3A3A3E08F828E83A3BB
:04304900A3A3F0222B
:0631D1008D4FAB07AA06BA
:1031D700908000E030E5079065787401F022906CEC
:1031E700801217758F538E528D518C50AE02AF03DC
:1031F7008E838F8263A201E552540744C0F583850D
:10320700538263A201AF4F121CBFE4FCFDFEE553DE
:10321700254FF553EE3552F552ED3551F551EC3555
:1032270050F550908040E550F0A3E551F0A3E552EA
:10323700F0A3E553F09080007420F0AF53AE52AD89
:0932470051AC50906C8012178DFF
:01325000225B
:063251008D4AAB07AA063E
:10325700908002E030E5079065787403F022906C67
:10326700841217758F4E8E4D8D4C8C4BAE02AF036B
:103277008E838F8263A201E54D540744D0F5838581
:103287004E8263A201AF4A121CBFE4FCFDFEE54E6D
:10329700254AF54EEE354DF54DED354CF54CEC35F3
:1032A7004BF54B908058E54BF0A3E54CF0A3E54D6B
:1032B700F0A3E54EF09080027420F0AF4EAE4DAD16
:0932C7004CAC4B906C8412178D85
:0132D00022DB
:022D7C008F4A7C
:102D7E00908001E030E5099065787402F07F0022C2
:102D8E00906C881217758F4E8E4D8D4C8C4B9066B5
:102D9E007B63A201E54D540744C8F583854E8263DB
:102DAE00A2017F06121CD5E54E2406F54EE4354DE4
:102DBE00F54DE4354CF54CE4354BF54B90657963A8
:102DCE00A201E54D540744C8F583854E8263A201E6
:102DDE00AF4A121CD5E4FCFDFEE54E254AF54EEE3B
:102DEE00354DF54DED354CF54CEC354BF54B9080A6
:102DFE004CE54BF0A3E54CF0A3E54DF0A3E54EF00A
:102E0E009080017420F0AF4EAE4DAD4CAC4B906C3B
:062E1E008812178DAF4A77
:012E2400228B
:1026B2009081E0E0F54A054A054A054A054A054A7D
:1026C200054A054A054A054A054A908010E0F54D3B
:1026D200A3E0F54EA3E0F54FA3E0F5509081E1E0D1
:1026E200F54A054A054A054A054A054A054A054A80
:1026F200054A054A054A908014E0F551A3E0F552D7
:10270200A3E0F553A3E0F554E553B54F08E554B5FE
:1027120050037F0022E4F54AE553540744E0F58371
:1027220085548263A20190637563A2017F08121D22
:102732000590637763A2019062AE63A2017F0612E5
:102742001C4D906375E0F54BA3E0F54CE4F54A901F
:102752006375E0702AA3E024F8F54AE55354074470
:10276200E0F58385548274082582F582E43583F589
:102772008363A20190637563A201AF4A121D05AE85
:102782004BE4FCFDE554254CF554E5533EF553ED81
:102792003552F552EC3551F551908014E551F0A3C4
:1027A200E552F0A3E553F0A3E554F09080007440A5
:0327B200F0AF4A3B
:0127B5002201
:101EFF009081E6E0F54A054A054A054A054A054A32
:101F0F00054A054A054A054A054A908028E0F54DDD
:101F1F00A3E0F54EA3E0F54FA3E0F5509081E7E085
:101F2F00F54A054A054A054A054A054A054A054A3A
:101F3F00054A054A054A90802CE0F551A3E0F55279
:101F4F00A3E0F553A3E0F554E4F54AE553B54F0A82
:101F5F00E554B55005C21F02206BE553540744F0FA
:101F6F00F58385548263A20190637563A2017F0894
:101F7F00121D05906375E0F54BA3E0F54CE54C455C
:101F8F004B70099080027410F07F0022906682E0FF
:101F9F00FFF46030906377E06F6003022032906649
:101FAF0083E0FF906378E06F7079906684E0FF9034
:101FBF006379E06F706D906685E0FF90637AE06FF4
:101FCF006031805F906377E0906682F0906378E095
:101FDF00906683F0906379E0906684F090637AE086
:101FEF00906685F090637BE0FFA3E0906349CFF0AC
:101FFF00A3EFF0906375E0702AA3E024F8F54AE5AB
:10200F0053540744F0F58385548274082582F58272
:10201F00E43583F58363A20190637563A201AF4A30
:10202F00121D05AE4BE4FCFDE554254CF554E5536C
:10203F003EF553ED3552F552EC3551F551AF50AEEB
:10204F004FAD4EAC4DAB54AA53A952A851D3121752
:10205F006440099080027410F07F002290802CE57C
:10206F0051F0A3E552F0A3E553F0A3E554F09080AF
:06207F00027440F0AF4ABC
:012085002238
:1021FC009081E3E0F54A054A054A054A054A054A35
:10220C00054A054A054A054A054A90801CE0F54DE9
:10221C00A3E0F54EA3E0F54FA3E0F5509081E4E088
:10222C00F54A054A054A054A054A054A054A054A3A
:10223C00054A054A054A908020E0F551A3E0F55285
:10224C00A3E0F553A3E0F554E4F54AE553B54F0A82
:10225C00E554B55005C220022352E553540744E817
:10226C00F58385548263A20190600463A2017F0E02
:10227C00121D1B906004E0F54BA3E0F54C90600C34
:10228C00E0FFF4604A90667BE0FEEF6E7079A3E0AD
:10229C00FF90600DE06F706F90667DE0FF90600EB8
:1022AC00E06F706390667EE0FF90600FE06F705798
:1022BC0090667FE0FF906010E06F704B906680E05E
:1022CC00FF906011E06F703FE4906013F080089015
:1022DC00601374FFF0D2D9906004E0702AA3E0245C
:1022EC00F2F54AE553540744E8F583855482740E9D
:1022FC002582F582E43583F58363A2019060046343
:10230C00A201AF4A121D1BAE4BE4FCFDE554254C5B
:10231C00F554E5533EF553ED3552F552EC3551F588
:10232C0051AF50AE4FAD4EAC4DAB54AA53A952A8C1
:10233C0051D31217645006E54C454B70099080013F
:10234C007410F07F0022908020E551F0A3E552F04C
:10235C00A3E553F0A3E554F09080017440F0AF4A2C
:01236C00224E
:042A64008E4F8F50B2
:102A6800908000E030E5079065787401F022906C62
:102A7800801217758F568E558D548C53E556FFE589
:102A8800555407FEE42FF552EE34C0F551855282B5
:102A9800F5837423F00552E552700205515351C76E
:102AA800F582855183740AF00552E552700205518A
:102AB8005351C790633E63A2018551838552826357
:102AC800A2017F06121CBF74062552F552E4355147
:102AD800F551854F8385508263A2018551838552C4
:102AE8008263A201121CA3E4FCFDFE906C80121705
:102AF8008112167BEF2408FFE43EFEE43DFDE43C32
:102B0800FC906C8012178D906C80E0908040F09063
:102B18006C81E0908041F0906C82E0908042F0906F
:0D2B28006C83E0908043F09080007420F0FA
:012B3500227D
:0A27B6008E4F8F508C518D528B53C3
:1027C000908000E030E5079065787401F022906C0D
:1027D000801217758F598E588D578C56E559FFE525
:1027E000585407FEE42FF555EE34C0F55485558254
:1027F000F5837423F00555E555700205545354C70D
:10280000F582855483740AF00555E5557002055428
:102810005354C790633E63A20185548385558263F8
:10282000A2017F06121CBF74062555F555E43554E8
:10283000F554854F8385508263A201855483855565
:102840008263A201121CA38F5AEF2555F555E4357A
:1028500054F554E553601785518385528263A20174
:1028600085548385558263A201AF53121CBFE55A7C
:1028700024082553F553FFE4FCFDFEE5592FF559D7
:10288000EE3558F558ED3557F557EC3556F5569069
:102890008040E556F0A3E557F0A3E558F0A3E559CD
:1028A000F09080007420F0AF59AE58AD57AC569000
:0528B0006C8012178D81
:0128B5002200
:062990008E4A8F4B8D4CB6
:10299600908000E030E5079065787401F022906C35
:1029A600801217758F528E518D508C4FE552FFE570
:1029B600515407FEE42FF54EEE34C0F54D854E8298
:1029C600F5837423F0054EE54E7002054D534DC751
:1029D600F582854D83EBF0054EE54E7002054D53AD
:1029E6004DC790633E63A201854D83854E8263A2E7
:1029F600017F06121CBF7406254EF54EE4354DF5D3
:102A06004D854A83854B8263A201854D83854E821F
:102A160063A201AF4C121CBF7408254CF54CFFE4B1
:102A2600FCFDFEE5522FF552EE3551F551ED3550D0
:102A3600F550EC354FF54F908040E54FF0A3E5504B
:102A4600F0A3E551F0A3E552F09080007420F0AFBA
:0D2A560052AE51AD50AC4F906C8012178DF8
:012A63002250
:0232D1008F6309
:1032D300908000E030E5079065787401F022906CEF
:1032E300801217758F678E668D658C64E567FFE5C1
:1032F300665407FEE42FFFEE34C09062B463A2016C
:10330300F5838F8263A201AF63121CBFE4FCFDFE51
:10331300E5672563F567EE3566F566ED3565F565B5
:10332300EC3564F564908040E564F0A3E565F0A3B3
:10333300E566F0A3E567F09080007420F0AF67AE18
:0B33430066AD65AC64906C8012178DC5
:01334E00225C
:0628B6008E4A8F4BAB05BA
:1028BC00908000E030E5079065787401F022906C10
:1028CC00801217758F518E508D4F8C4EE551FFE550
:1028DC00505407FEE42FF54DEE34C0F54C854D8277
:1028EC00F5837423F0054DE54D7002054C534CC730
:1028FC00F582854C83EBF0054DE54D7002054C904F
:10290C00633E63A201854C83854D8263A2017F06E1
:10291C00121CBF7406254DF54DE4354CF54C534C4B
:10292C00C7E54A854D82854C83F0054DE54D700217
:10293C00054C534CC7F582854C83E54BF0054DE5B2
:10294C004D7002054C534CC7E551240AF551E43542
:10295C0050F550E4354FF54FE4354EF54E90804030
:10296C00E54EF0A3E54FF0A3E550F0A3E551F09050
:10297C0080007420F0AF51AE50AD4FAC4E906C80D7
:03298C0012178D92
:01298F002225
:0A391C00E4FEEEC39F50030E80F896
:01392600227E
:10387000A2AF9237C2AF438E2075D2028F828E8361
:0C388000E0FFE4F5D2538EDFA23792AFD8
:01388C002219
:1037C400E5D220E0FBA2AF9237C2AF43D2028F8290
:1037D4008E83EDF075D25063D250A23792AFE5D20A
:0337E40020E0FBE7
:0137E70022BF
:10334F00E4FDED2401FFE433FE12387074362DF5E1
:10335F0082E43463F583EFF00DBD3FE6E4FDED2429
:10336F007FFFE433FE123870742D2DF582E4346143
:10337F00F583EFF0742D2DF582E43461F583E07061
:10338F001B742D2DF582E43461F5837420F0742EB7
:10339F002DF582E43461F583E4F080040DBD80BE29
:1033AF00E49061ACF0FDEDFF7E0012387074AD2D2E
:0D33BF00F582E43461F583EFF00DBDFEE909
:0133CC0022DE
:02375E008B4F8F
:10376000A2AF9237C2AF85A25053A2FE8E838F8242
:1037700005A28C838D827409121D49E54F53A2FE68
:1037800043A220121D4B53A2DF8550A2A23792AF55
:01379000FF39
:013791002215
:10388D00A2AF9237C2AF8C838D82EF121D4943A236
:0C389D0020121D4B53A2DFA23792AFFF98
:0138A90022FC
:0237E8008F4A06
:1037EA00A2AF9237C2AFE4F5838D827406121D49E7
:1037FA00E54A43A220121D4B53A2DFA23792AF7FA4
:01380A0001BC
:01380B00229A
:02380C008F4AE1
:10380E00A2AF9237C2AFE4F5838D82740A121D49BE
:10381E00E54A43A220121D4B53A2DFA23792AF7F7F
:01382E000198
:01382F002276
:101B7200A907E7FFA805EF93C3966008403B74FCF2
:101B82002FFF80F00F08EF93C3966008402B74FB81
:101B92002FFF80E00F08EF93C3966008401B74FA92
:101BA2002FFF80D00F08EF93D3966008400B74F993
:101BB2002FFF80C01F1F1F1F1FEF54FEF80303F7E4
:101BC200E893FC08E893FD08E893FE08E893FF22F7
:101BD20009E993C39D6008402974FB29F980F10942
:101BE200E993C39E6008401A74FA29F980E209E970
:101BF20093D39F6008400B74F929F980D3191919FE
:101C02001919E9C313C313FF22740093F8ECC398A4
:101C12004024701F740193F8EDC398401970147436
:0E1C22000293F8EEC398400E7009740393F815
:101C3000EFC39840037F00227F0122EDF8E6F00811
:101C4000A3DFFA22EDF8E0F608A3DFFA22E0A363AF
:101C5000A201F0A363A201DFF475A2002263A20136
:101C6000F0A363A20122E0A363A201F0A363A20197
:101C7000E0A363A201F0A363A201E463A201F0A3C5
:101C800063A201DFE175A20022E0A363A2016DFE61
:101C9000936CFDEE058393FC158363A201DFEA7567
:101CA000A200227F00E493A363A201F00F600CA3C3
:101CB000E583C2E3F58363A20180EA75A20022E016
:101CC000A363A201F0A3E583C2E3F58363A201DF6E
:101CD000EE75A20022E0A363A201F0A3E583C2E4B3
:101CE000D2E3F58363A201DFEC75A20022E0A363D7
:101CF000A201F0A3E58344F8C2E5F58363A201DF06
:101D0000EC75A20022E583C2E3F583E0A363A201A0
:101D1000F0A363A201DFEE75A20022E583C2E4D244
:0A1D2000E3F583E0A363A201F0A342
:101D2A0063A201DFEC75A20022E58344F8F583E0A3
:101D3A00A363A201F0A363A201DFEE75A20022F958
:101D4A0022C002C004C00612FFF0D006D004D0029E
:011D5A002266
:101911000A53656E643A20000A446174612066725C
:101921006F6D207365727665723A000A43524320E7
:101931006572726F722120000A53796E63204572BD
:10194100726F722120000A526563204F4B212000E3
:101951000A5374617274207472616E736D697420BC
:10196100000008040C020A060E0109050D030B070D
:101971000F00112332465765748C9DAFBECADBE957
:10198100F810013322564775649C8DBFAEDACBF94E
:10199100E82130021367764455ADBC8E9FEBFAC83F
:1019A100D93120120377665445BDAC9E8FFBEAD82E
:1019B100C94253617004152736CEDFEDFC8899AB1F
:1019C100BA5243716014053726DECFFDEC9889BB0E
:1019D100AA6372405125340617EFFECCDDA9B88AFF
:1019E1009B7362504135241607FFEEDCCDB9A89AEE
:1019F1008B8495A7B6C2D3E1F008192B3A4E5F6DDF
:101A01007C9485B7A6D2C3F1E018093B2A5E4F7DCD
:101A11006CA5B48697E3F2C0D129380A1B6F7E4CBE
:101A21005DB5A49687F3E2D0C139281A0B7F6E5CAD
:101A31004DC6D7E5F48091A3B24A5B69780C1D2F9E
:101A41003ED6C7F5E49081B3A25A4B79681C0D3F8D
:101A51002EE7F6C4D5A1B082936B7A48592D3C0E7E
:101A61001FF7E6D4C5B1A092837B6A58493D2C1E6D
:101A71000F0089129B24AD36BF48C15AD36CE57E55
:101A8100F78108931AA52CB73EC940DB52ED64FFDC
:101A910076028B109926AF34BD4AC358D16EE77CCC
:101AA100F5830A9118A72EB53CCB42D950EF66FDBC
:101AB10074048D169F20A932BB4CC55ED768E17AAC
:101AC100F3850C971EA128B33ACD44DF56E960FB9C
:101AD10072068F149D22AB30B94EC75CD56AE3788C
:101AE100F1870E951CA32AB138CF46DD54EB62F97C
:101AF1007008811A932CA53EB740C952DB64ED767C
:101B0100FF89009B12AD24BF36C148D35AE56CF75B
:101B11007E0A8318912EA73CB542CB50D966EF744B
:101B2100FD8B029910AF26BD34C34AD158E76EF53B
:101B31007C0C851E9728A13AB344CD56DF60E9722B
:101B4100FB8D049F16A920BB32C54CD75EE168F31B
:101B51007A0E871C952AA338B146CF54DD62EB700B
:101B6100F98F069D14AB22B930C74ED55CE36AF1FB
:011B710078FB
:1038B00052668D00000000000000000000000000C3
:0538C000000000000003
:10385200906A67E06FFC901A7293FE906A66E06E5F
:0D386200A3F0AF04EF90197293906A66F026
:01386F002236
:0100210022BC
:1038F800EF540F90196293FEC454F0FEEFC4540FB6
:04390800932EFF22D9
:1037920030152CE4906475F0E51424FEFFA3F0903C
:1037A200667AE0906477F0A37408F090696663A289
:1037B2000190647963A201121C4DC2157F01227F20
:0237C2000022E3
:10368A00C237E4FEE51364056032BF7E07D205E463
:10369A00F50FF513EF30E7074308010513800653CA
:1036AA0008FEE4F513050FE50FB40808850816D2DD
:1036BA0037E4F50FE50825E0F508800CEF30E7055B
:1036CA00D205A23722E4F513EF25E0FF0EBE08B4B7
:0236DA00A23715
:0136DC0022CB
:1034B500E4FEE50E25E0F50EEF30E736430E01207C
:1034C5003733050DE50DB4052CE4F50D0512E512B0
:1034D500B40817050CE50CAC0B7002050B14F5824E
:1034E5008C83E50EF00515E4F512E50E25E0F50EE5
:1034F5008003E4F50D0512E512B40817050CE50C7B
:10350500AC0B7002050B14F5828C83E50EF00515E6
:0D351500E4F512EF25E0FF0EEE640870955E
:013522002286
:1038300075487E7540A0C208D20FC215D22FC213A0
:10384000C202C214D201C211E4F53FF53CC291C2DA
:023850009022C4
:04249F008E4B8F4C85
:1024A300906A66E0906C8EF0906A67E0906C8FF0B3
:1024B300E4F515F50D906A66F0A3F0AB4CAA4B75E5
:1024C3000B69750CE6301025850C82850B83740A25
:1024D300F0050CE50C7002050BF582850B8374AADD
:1024E300F0050CE50C7002050B05150515850C822E
:1024F300850B83747EF0050CE50C7002050B051546
:10250300E4F512906C8CF0906C8CE0C39D50498B79
:10251300828A83E0FF1238F8906C8DEFF0906A673F
:10252300E06F906C8DF0E0FF901A7293FE906A66F4
:10253300E06EA3F0EF90197293906A66F00BEBAE26
:102543000270010A14F5828E83E0FFC2371234B59C
:10255300906C8CE004F080AF906A67E0FF1238F86B
:10256300C2371234B5906A66E0FF1238F8C23712E8
:1025730034B5D2377F7E1234B5D237E4FF1234B587
:10258300D2027C697DE68C0B8D0C3024097E197F89
:1025930011AB151227B6906C8EE0906A66F0906CC2
:0625A3008FE0906A67F072
:0125A900220F
:103636008F4A20022130110E7E697F26E54A24FC3E
:10364600FD12249F800C7E637F79E54A24FCFD12DF
:10365600249FC211801C201119854A11D211906332
:103666007963A20190692663A201E54A24FCFF1250
:103676001C4D30240B7E197F19E4FBFDFC1227B686
:04368600854A4A2205
:102CC700E4FF0F2405F582E43461F5837408F00FFF
:102CD70074052401F582E43461F583E4F07C667DB4
:102CE70092FEED1DAA0470011CF5828A83E0FBAAFF
:102CF700070F74052AF582E43461F583EBF00EBE05
:102D070004E07C667D96E4FEED1DAA0470011CF5C7
:102D1700828A83E0FBAA070F74052AF582E43461EF
:102D2700F583EBF00EBE04E07C667D9AE4FEED1DB4
:102D3700AA0470011CF5828A83E0FBAA070F7405B9
:102D47002AF582E43461F583EBF00EBE04E07C667D
:102D57007D9EE4FEED1DAA0470011CF5828A83E0C6
:102D6700FBAA070F74052AF582E43461F583EBF0BB
:042D77000EBE04E0A8
:012D7B002235
:1038C600D201D291D208E4F514F513906A67F0900C
:0C38D6006A66F0F50F750969750A662234
:10236D00200803022467E53E5438653A70030224C1
:10237D009EE53A24085438F53A131313541F242AB2
:10238D00F8E6F51020053020072DFF12368A50D6BD
:10239D00AF161238F8123852050AE50AAE09700266
:1023AD00050914F5828E83E516F00514E514D39412
:1023BD004040B3D20780AFE514D394024005200707
:1023CD0002D215C208C205E4F528D22FC291906A37
:1023DD0067E0FF906A66E04F6037C21530240D7ECE
:1023ED00197F2C7C697D66AB141227B69066971207
:1023FD001775E47B01FAF9F812167B9066971217A0
:10240D008D906966E0704E20074BC22F1238C68042
:10241D0044906966E07014C2153024397E197F39F5
:10242D007C697D66AB141227B6802A30240D7E1987
:10243D007F477C697D66AB141227B690668F1217A5
:10244D0075E47B01FAF9F812167B90668F12178DE1
:10245D00E4906A69F0C207022373202F34E52AB491
:10246D007E0F300308E4F528D22FC203221238C69E
:10247D0022E52AB54016200613D2019066A0E0FF92
:10248D00A3E0906924CFF0A3EFF0C209E4F528D2C0
:02249D002F22EC
:1025AA0030302DC3E5439546FFE5429545FED3EF0E
:1025BA009440EE940040197B087D40AF46AE451228
:1025CA002990E5462440FFE43545540FF5458F46EA
:1025DA00201A05D291D2902230190AC2199067A204
:1025EA00E0600214F0300F0312236D301366E53FEA
:1025FA00653C603BE53F24085438FFE53C54386F9E
:10260A0070030226B1E51570030226B1050CE50C2C
:10261A00AC0B7002050B14F5828C83E0FEE53F13C8
:10262A001313541F2432F8A6068F3F151580C5C20E
:10263A0090C213C202906693121775E47B01FAF9ED
:10264A00F812167B90669312178DD214D2B1E490C9
:10265A0067A2F022200850300245E53F653C7047EA
:10266A0030240D7E197F517C697D66AB141227B622
:10267A00050CE50CAE0B7002050B14F5828E83E097
:10268A00FFE53F131313541F2432F8A607E53F242E
:10269A00085438F53F1515D213D2907599AA2230ED
:0826AA001105AF1112363622B2
:0B392700301405C2147F01227F002233
:03001E00C2AE224D
:102086003E2A2C312CCFE0F0E0ECE5F2F0FB20E02C
:10209600F1E8EDF5F0EEEDEDEEE3EE20EFEEF0F229
:1020A600E02E0A003E4C2C4930312C256C752CD183
:1020B600EAEEF0EEF1F2FC20EEE1ECE5EDE02C3597
:1020C600302C3130302C3330302C3630302C31320D
:1020D60030302C323430302C343830302C393630E5
:1020E600302C31393230302C33383430302C3537CF
:1020F6003630302C3131353230300A003E422C49F0
:1021060030322C2562752CD3EFF0E0E2EBE5EDE8FA
:10211600E520EFEEF2EEEAEEEC20EFF0E820EFE558
:10212600F0E5E4E0F7E520285254532D43545329B3
:102136000A003E532C4930332C2562752CC7E0E447
:10214600E5F0E6EAE020F1F2E0F0F2E020EFE5F07B
:10215600E5E4E0F7E8282A3130ECF1290A003E42AE
:102166002C4930342C2562752CD0E5E6E8EC20EFBE
:10217600E5F0E5E4E0F7E8203720E1E8F20A003E82
:10218600422C4930352C2562752CCFE5F0E5E4E08C
:10219600F7E020F120EAEEEDF2F0EEEBFCEDFBECE1
:1021A60020E1E8F2EEEC0A003E422C4930362C25BE
:1021B60062752CCAEEEDF2F0EEEBFCEDFBE920E1E8
:1021C600E8F2202D20F7E5F2EDEEF1F2FC0A003CF4
:1021D60021003C4930313D003C4930323D003C490C
:1021E60030333D003C4930343D003C4930353D00FC
:0621F6003C4930363D00BB
:0100220022BB
:030023000230D0D8
:0730D000C0E0C0D075D0186C
:1030D70030984DC298AF99E4FEE52825E0F528EF32
:1030E70030E7020528EF25E0FF302F19E52865486E
:1030F7006006E52865407024753A00753E0085280E
:103107002AC22F8017053EE53E5407700F533E3FF6
:10311700E53E131313541F242AF8A6280EBE08B938
:10312700309920C299E53F653C6018E53C131313BD
:10313700541F2432F8E6F529F5997408253CF53C27
:05314700533C3FD2AF34
:05314C00D0D0D0E032FC
:102F41007BFF7A20798612136B906A6CE0FEA3E016
:102F5100FFC3E49FFFE49EFEAB07FA3395E0F9F867
:102F61007F007E8C7D0A7C001216C48F558E548D95
:102F7100538C527BFF7A2079AA12136B7BFF7A2143
:102F81007902A212E433F55212136B7BFF7A217995
:102F91003890669FE0F55212136B7BFF7A217964BA
:102FA100A22EE433F55212136B7BFF7A217985A2AD
:102FB10028E433F55212136B7BFF7A2179AEA22BF1
:082FC100E433F55212136B22F8
:102C00007E217FD5123151EF4E70037F01227E214C
:102C10007FD8123151EF4E6023123523A804A90545
:102C2000AA06AB077F007E8C7D0A7C001216C412B8
:102C30001756906A6CEEF0A3EFF0800A906A6C74FD
:102C4000FFF0A374B8F07E217FDE123151EF4E60A9
:102C50000C1238E2EF24D024FF92128002C2127EBE
:102C6000217FE4123151EF4E600A12352390669FA6
:102C7000EFF08005E490669FF07E217FEA123151EB
:102C8000EF4E600C1238E2EF24D024FF922E800227
:102C9000C22E7E217FF0123151EF4E600C1238E2CD
:102CA000EF24D024FF92288002C2287E217FF612D2
:102CB0003151EF4E600C1238E2EF24D024FF922BFA
:072CC0008002C22B7F0022FD
:10304D00C22AC22DC229C232E4F544906A70F0F54D
:10305D0041F56BC227C22EC22BC228C234C212F553
:10306D003BD235906A6C74FFF0A374B8F0122C004B
:10307D00906A717401F0C2ADE4F5C9D2CDD2CCC263
:10308D00C9C2CAF5CDF5CC906A6CE0F5CBA3E0F5DD
:10309D00CA85CBCD85CACCE4F59830280C202E09F5
:1030AD005387BFD29FD29E8002D29E438740C29F3C
:1030BD00C2ACC298C29975B81075B710D2CAD29C5D
:0330CD00D2AC2260
:102EC100020869E493A3F8E493A34003F68001F2B6
:102ED10008DFF48029E493A3F85407240CC8C33312
:102EE100C4540F4420C8834004F456800146F6DFE1
:102EF100E4800B01020408102040809038AAE47E8F
:102F0100019360BCA3FF543F30E509541FFEE493D5
:102F1100A360010ECF54C025E060A840B8E493A39C
:102F2100FAE493A3F8E493A3C8C582C8CAC583CAC7
:102F3100F0A3C8C582C8CAC583CADFE9DEE780BE7F
:0138C5000002
:10166500C5F0F8A3E028F0C5F0F8E5821582700210
:061675001583E038F022AD
:0D167B00EF2BFFEE3AFEED39FDEC38FC22BE
:1016880075F008758200EF2FFFEE33FECD33CDCC19
:1016980033CCC58233C5829BED9AEC99E58298409C
:1016A8000CF582EE9BFEED9AFDEC99FC0FD5F0D679
:1016B800E4CEFBE4CDFAE4CCF9A88222B800C1B9A3
:1016C8000059BA002DEC8BF084CFCECDFCE5F0CBE1
:1016D800F97818EF2FFFEE33FEED33FDEC33FCEB1A
:1016E80033FB10D703994004EB99FB0FD8E5E4F9D5
:1016F800FA227818EF2FFFEE33FEED33FDEC33FCC2
:10170800C933C910D7059BE99A4007EC9BFCE99AB5
:10171800F90FD8E0E4C9FAE4CCFB2275F010EF2FFA
:10172800FFEE33FEED33FDCC33CCC833C810D707FA
:101738009BEC9AE899400AED9BFDEC9AFCE899F835
:0E1748000FD5F0DAE4CDFBE4CCFAE4C8F922C8
:0E175600C3E49FFFE49EFEE49DFDE49CFC22A4
:10176400EB9FF5F0EA9E42F0E99D42F0E89C45F0DB
:011774002252
:0C177500E0FCA3E0FDA3E0FEA3E0FF22E7
:0C178100E0F8A3E0F9A3E0FAA3E0FB22EB
:0C178D00ECF0A3EDF0A3EEF0A3EFF022CF
:10179900A8828583F0D083D0821217B01217B012B5
:1017A90017B01217B0E473E493A3C583C5F0C583DA
:1017B900C8C582C8F0A3C583C5F0C583C8C582C89A
:0117C90022FD
:10130900E55E2452F8E6055E22784F303E027852B7
:10131900E475F0011218710217CA2037EB7F2ED23B
:10132900378018EF540F2490D43440D4FF303B0B4E
:10133900EF24BFB41A0050032461FFE55F60021572
:101349005F0562E56270020561303E0D784FE47514
:10135900F001121871EF0218100236DD7403D23E43
:101369008003E4C23EF55E8B4F8A508951E4F55FF4
:10137900F561F562E55F60077F2012134480F5751A
:1013890060FFC238C237C239C23AC23CC23DC23F0D
:10139900121312FF700D303E057F00121355AF6214
:1013A900AE6122B4255FC2D5C23B121312FF24D00D
:1013B900B40A00501A75F00A785F30D50508B6FFEF
:1013C9000106C6A426F620D5047002D23A80D92493
:1013D900CFB41A00EF5004C2E5D23B021555D238FA
:1013E90080C6D23780C0D23980BCD2D580BAD23C2F
:1013F90080B47F201213442039077401B55F00407F
:10140900F1121309FF12134402137DD23FD23D801A
:1014190095121309FB121309FA121309F94A4B70B1
:101429000679267A167BFF20392EE55F602A7E0031
:101439008E827583001217E360060EEE656070F008
:10144900C2D5EBC0E0EAC0E0E9C0E0EE12159CD0DD
:10145900E0F9D0E0FAD0E0FB1217CAFF60AAEBC0AE
:10146900E0EAC0E0E9C0E0121344D0E02401F9D079
:10147900E03400FAD0E0FBE5600460DCD560D98097
:10148900877BFF7A157998D239809C791080027907
:1014990008C23DC23F8008D2D5790A8004790AC2C0
:1014A900D5E560047002F560E4FAFDFEFF12130948
:1014B900FC7B08203813121309FD7B1030370A1200
:1014C9001309FE121309FF7B20EC3382D592D55004
:1014D90013C3E43037069FFFE49EFEE42038039DE2
:1014E900FDE49CFCE4CBF8C238EC700CCFCECDCC3B
:1014F900E824F8F870F38017C3EF33FFEE33FEEDFD
:1015090033FDEC33FCEB33FB994002FB0FD8E9EBDD
:10151900303805F8D0E0C448B238C0E00AEC4D4E86
:101529004F78207B0070C2EAB5600040BCC0E01271
:10153900159ED0F0D0E0203804C4C0E0C4B238C051
:10154900F012132DD0F0D5F0EB02137D1218D01440
:101559001A5314945813EB4C13E74214984F14A0E0
:0F1569004414A04914004314A655148A46148A4A
:1015780045148A4716465013EF2D13F32E14162BD5
:1015880013F723141420162F2A13AF480000140E43
:101598003F3F3F00790AA2D5203A14303C09B910E0
:1015A800020404B9080104A2D5203D025001042018
:1015B80039689239B55F005034C0E07F20303A195D
:1015C8007F30A239723D723C500F1215F5C239C2F4
:1015D8003DC23CC23F7F30800F303C03E9C0E0127F
:1015E8001344303C03D0E0F9D0E0B55FCC303C1771
:1015F8007F30B9100C1213447F58303B077F788036
:1016080003B908031213443039057F2D0213447FB0
:1016180020203FF87F2B203DF322923980CF286E7F
:10162800756C6C2900D2381213093038F8C2387832
:101638005F30D50108F60213AF2D504349581213F5
:10164800092403B405004001E490164193121335B0
:0D165800743A121335D23A755F04021494EF
:101D5B008B4A8A4B894CE4F556F555F554F553F5FA
:101D6B0051F552E54E454F454D6012EBC0E0EAC0D0
:101D7B00E0E9C0E0AB4DAA4EA94F121881AB4A0562
:101D8B004CE54CAA4B7002054B14F91217CAF557C8
:101D9B00C394094007E557D3940D40E1E557642000
:101DAB0060DBE557B42D054352038016E557B42B82
:101DBB0005435201800C74FF254CF54C74FF354BD9
:101DCB00F54BE55060046410703FAB4AAA4BA94C2D
:101DDB001217CA64306009E550702E75500A8029BD
:101DEB009000011217E3FF64786004EFB4581343BB
:101DFB0052017550107402254CF54CE4354BF54BE4
:101E0B008007E5507003755008AB4A054CE54CAAAA
:101E1B004B7002054B14F91217CAF557C394614066
:101E2B000AE557D3947A50035357DF74D02557F5EF
:101E3B0057C3940A400CE5579411406D74F925571C
:101E4B00F557E557D39550506043520185565B8546
:101E5B00555A855459855358AF507E00E4FCFDAB61
:101E6B0056AA55A954A853121822C8ECC8C9EDC9D3
:101E7B00CAEECACBEFCBE4FCFDFEEB2557F556EED5
:101E8B003AF555ED39F554EC38F553AF56AE55AD33
:101E9B0054FCAB5BAA5AA959A858D3121764500328
:101EAB00021E14435204021E14E55220E003E48088
:101EBB002DE54E454F454D601EAB4AE54C24FFF9D1
:101ECB00E54B34FFFAEBC0E0EAC0E0E9C0E0AB4D14
:101EDB00AA4EA94F121881E55230E20774FFFFFE9C
:101EEB00FDFC22E552AF56AE55AD54AC5330E10379
:041EFB000217562252
:1017CA00BB010689828A83E0225002E722BBFE021D
:0917DA00E32289828A83E4932250
:1017E300BB010CE58229F582E5833AF583E02250BB
:1017F30006E92582F8E622BBFE06E92582F8E22205
:0D180300E58229F582E5833AF583E493221E
:10181000BB010689828A83F0225002F722BBFE01B7
:02182000F322B1
:10182200E88FF0A4CC8BF0A42CFCE98EF0A42CFC65
:101832008AF0EDA42CFCEA8EF0A4CDA8F08BF0A4E3
:101842002DCC3825F0FDE98FF0A42CCD35F0FCEB42
:101852008EF0A4FEA9F0EB8FF0A4CFC5F02ECD3907
:0F186200FEE43CFCEAA42DCE35F0FDE43CFC2274
:10187100FAE6FB0808E6F925F0F618E6CA3AF62278
:10188100BB011A89828A83D0F0D0E0F8D0E0F9D088
:10189100E0FAD0E0FBE8C0E0C0F00218FF5016E922
:1018A100F8D083D082D0E0F9D0E0FAD0E0FBC0825A
:1018B100C0830218F6BBFE16E9F8D083D082D0E0CF
:0F18C100F9D0E0FAD0E0FBC082C0830219082200
:1018D000D083D082F8E4937012740193700DA3A3A7
:1018E00093F8740193F5828883E4737402936860BB
:0618F000EFA3A3A380DFBB
:0918F600EBF608EAF608E9F62217
:0918FF00EBF0A3EAF0A3E9F022EA
:09190800EBF208EAF208E9F22210
:00000001FF
